:020000020000FC
:100000000FC09AC09DC09FC0A4C0A4C09AC09AC08F
:04001000A3C0A1C028
:10002000F894F0E0E0E600E00193E03AE9F70EE949
:100030000DBF00E810E006BD16BD00E00BBF00E0FC
:1000400009BF00E005BB00E60ABF0EE008BF03E2FF
:1000500008BB0DE107BB02E005BF00E002BF00E006
:100060000FBD05E003BF00E006BF00E009BD00E0F2
:1000700008BD00E007B900E003B900E006B900E000
:1000800004BB00E808B9A89504B7077F04BF01B511
:10009000006101BD0EE401BD00E40BBF02E009BF39
:1000A000D2E1C0E5F5E0ECED05E0502E00EA402E8F
:1000B00090E07894A89590FFFDCF9E7FB0E0A0E0FF
:1000C0001196B19BFDCF1B2F0A2F31E020EE8894B3
:1000D000020B130B08F42FC01B2F0A2F39E020E668
:1000E0008894020B130B08F026C03B2E2A2E132DEA
:1000F000022D88940409150930F40095109520E02C
:100100000894021F121F30E020E18894020B130BA9
:1001100028F0532C422C75E29D7F01C0000091FD18
:1001200009C0B32DA22DF894C09A00001197E9F7E9
:10013000C09878940000BECFFFB69160FFBE1895BE
:10014000189518951895FFB67A9509F49260FFBE38
:10015000189518951895189518954F935F936F9368
:10016000551B441B61E110F4400F511F57954795F3
:10017000379527956A95B9F75F934F933F932F93E0
:100180000F911F912F913F916F915F914F91089522
:100190004F935F936F934427552760E1000F111F22
:1001A000441F551F4217530718F00395421B530B6A
:1001B0006A95A1F75F934F932F913F916F915F9154
:1001C0004F9108951F932F9310EF25E0A8952A953E
:1001D000E9F71A95D1F70A95B9F72F911F9108956C
:00000001FF
